:1000000014C019C018C017C016C015C014C013C042
:1000100012C011C010C00FC00EC00DC00CC00BC06C
:100020000AC009C008C007C006C011241FBECFED1A
:10003000CDBFF6D026C1E4CF0F931F93FC01213032
:10004000310531F5101611060CF042C051E001C027
:10005000550F4A95EAF720E030E088B3452F482B4A
:10006000CF01022E02C0959587950A94E2F7817020
:100070009927062E02C0880F991F0A94E2F7842B55
:1000800088BB18BA2F5F3F4F2017310731F720C0C8
:1000900001501109EAF081E001C0880F4A95EAF7A2
:1000A00028B3982F922B9F01002E02C035952795DB
:1000B0000A94E2F721703327062E02C0220F331F65
:1000C0000A94E2F7292B28BB18BA0150110940F70E
:1000D0001F910F910895EF92FF920F931F93CF936B
:1000E000DF93EA0143E050E09A01281B390BC90174
:1000F00021E030E0F90102C0EE0FFF1F8A95E2F720
:10010000CF01809590958F709927461B570B02C0A1
:10011000220F331F4A95E2F722953295307F32271E
:10012000207F3227280F391F7901FF242097D9F427
:1001300018BA00E110E021E030E042E050E061E078
:1001400070E080E09E2D78DF81E088BB18BA21E066
:1001500030E045E050E064E070E080E090E06CDF8B
:1001600088E088BB3BC0C130D105D1F418BA00E1AA
:1001700010E021E030E042E050E061E070E0C701D3
:100180005BDF81E088BB18BA21E030E045E050E059
:1001900064E070E080E090E04FDF88E088BB39C029
:1001A000C230D105D9F418BA00E110E021E030E006
:1001B00045E050E064E070E080E09E2D3DDF88E0A7
:1001C00088BB18BA21E030E042E050E061E070E026
:1001D00080E090E031DF81E088BB1BC02397C9F449
:1001E00018BA00E110E021E030E045E050E064E0C2
:1001F00070E0C70121DF88E088BB18BA21E030E059
:1002000042E050E061E070E080E090E015DF81E0E6
:1002100088BBDF91CF911F910F91FF90EF900895D0
:100220008FE387BB812C912CA82CB92CC82CD92CFE
:10023000E82CF92C23C0A701BE01C8014CDF83ECD8
:1002400099E00197F1F700C000002196C430D10574
:1002500091F787EA91E60197F1F700C000000F5F80
:100260001F4F0430110519F0CC2DDD2DE4CF9FEF89
:10027000E91AF90A84E0E816F104D1F20A2D1B2DDF
:06028000F3CFF894FFCF5C
:00000001FF
